:100000000C9434000C9449000C9449000C94490061
:100010000C9449000C9449000C9449000C9449003C
:100020000C9449000C9449000C9449000C9449002C
:100030000C9449000C9449000C9449000C9449001C
:100040000C9449000C9449000C9449000C9449000C
:100050000C9449000C9449000C9449000C944900FC
:100060000C9449000C94490011241FBECFEFD8E036
:10007000DEBFCDBF11E0A0E0B1E0E4E8FAE002C0ED
:1000800005900D92A433B107D9F70E949F010C94FB
:1000900040050C940000549A529A84B18E6184B940
:1000A000539A08955C9A00000000000000000000D0
:1000B00000005C980895CF93DF9395B1917E95B938
:1000C00045B1C82FD0E09E01207F3070C9019595C1
:1000D00087959595879595958795842B85B90E94E9
:1000E000520085B1817E85B925B1CE018F709070A7
:1000F000EC01CC0FDD1FAE01422B45B90E9452002E
:10010000DF91CF9108958FE39FE10197F1F700C050
:10011000000080E008951F93182F0E948300882319
:10012000E4F35A985B98812F0E945B001F91089519
:100130000E944B008FE59AEE0197F1F700C0000096
:100140005A985B9885B1817E85B985B1866085B9FD
:100150000E9452008FE19EE40197F1F700C0000079
:100160000E9452008FE99FE00197F1F700C0000064
:100170000E94520085B1817E85B92A9A8FE99FE05D
:100180000197F1F700C000000E9452008FE39FE149
:100190000197F1F700C0000088E20E948B008FE316
:1001A0009FE10197F1F700C0000081E00E948B0001
:1001B0008FE39FE10197F1F700C0000082E00E9409
:1001C0008B008FE39FE10197F1F700C000008EE004
:1001D0000E948B0008951F93182F0E94830088238C
:1001E000E4F35A9A5B98812F0E945B001F91089557
:1001F000CF93DF93EC018881882331F021960E9410
:10020000EB0089918823D9F7DF91CF910895EF9280
:10021000FF920F931F93CF93DF93082F192F862FF1
:10022000880F880F880F80640E948B00E02EE70102
:100230007E01F12EE70118E089910E94EB00115038
:10024000D9F7DF91CF911F910F91FF90EF90089513
:1002500088E091E064E00E94070180E191E060E0C5
:100260000E94070180E80E948B0008951F93CF939E
:10027000DF9310E0C0E0D1E0CE01612F0E940701C2
:100280001F5F1830C9F780E80E948B00DF91CF9183
:100290001F910895CF93DF93EC018881882331F07B
:1002A00021960E94EB0089918823D9F7DF91CF91A5
:1002B00008950E9483008823E4F30E948300089538
:1002C0001F930E945901182F88E191E067E00E9476
:1002D0000701812F80680E948B001F910895109262
:1002E0008000109281000895209A289A2AE12A9588
:1002F000F1F700C028982098189BFECF1092850037
:1003000010928400E1E8F0E0808182608083E4E87C
:10031000F0E006C0808191812AEE8136920710F4C8
:100320001899F8CF809184009091850010928100F7
:1003300064E770E00E943D02862F972F0895AF92E8
:10034000BF92CF92DF92EF92FF920F931F93DF93B2
:10035000CF93CDB7DEB760970FB6F894DEBF0FBE70
:10036000CDBF0E9405020E9498000E946F018E017D
:100370000F5F1F4FEE24FF246894E4F80F2EF0E285
:10038000CF2EF1E0DF2EF02D0F2EF1E3AF2EF1E0B6
:10039000BF2EF02D0E9474012DB73EB7285030407B
:1003A0000FB6F8943EBF0FBE2DBFEDB7FEB7319626
:1003B000ADB7BEB712961C930E931197F382E282EB
:1003C000D582C482978386830E9451022DB73EB79F
:1003D000285F3F4F0FB6F8943EBF0FBE2DBF80E899
:1003E0000E948B00C8010E94F800C8010E942602EA
:1003F000C5010E9426028FEF93ECA9E08150904046
:10040000A040E1F700C00000C5CF1092C50087E60C
:100410008093C400E0ECF0E080818D7F808386E0F3
:100420008093C20088E18093C10008951F93182F24
:100430008A3019F48DE00E941602E0ECF0E0808131
:1004400085FFFDCF1093C6001F910895CF93DF93D2
:10045000EC018881882331F021960E94160289914F
:100460008823D9F7DF91CF910895E0ECF0E0808107
:100470008823ECF78091C6000895AA1BBB1B51E1AD
:1004800007C0AA1FBB1FA617B70710F0A61BB70B04
:10049000881F991F5A95A9F780959095BC01CD01A9
:1004A0000895AEE0B0E0E7E5F2E00C9417050D89A1
:1004B0001E898F89988D26E02C831A83098397FFE4
:1004C00002C080E090E801979E838D839E01255EA7
:1004D0003F4FCE010196698D7A8DA9010E9482025B
:1004E0004D815E8157FD0AC02F8138854217530721
:1004F0000CF49A01020F131FF80110822E96E4E00B
:100500000C943305ACE0B0E0E8E8F2E00C940905A7
:100510006C011B018A01FC0117821682838181FF15
:10052000D1C12E010894411C511CF6019381F101A7
:1005300093FD859193FF81911F01882309F4BEC12A
:10054000853239F493FD859193FF81911F018532A6
:1005500029F490E0B6010E947F04E7CFEE24FF2447
:1005600020E02032B0F48B3269F08C3228F48032F3
:1005700051F0833271F40BC08D3239F0803349F47D
:1005800021602CC02260246029C0286027C020611F
:1005900025C027FD2CC0382F30533A3098F426FF61
:1005A00008C08E2D880FE82EEE0CEE0CE80EE30E40
:1005B00015C08F2D880FF82EFF0CFF0CF80EF30ED0
:1005C00020620CC08E3221F426FD78C1206406C062
:1005D0008C3611F4206802C0883649F4F10193FD8D
:1005E000859193FF81911F01882309F0BACF982F3D
:1005F0009554933018F09052933028F40C5F1F4FAD
:10060000FFE3F9830DC0833631F0833771F0833512
:1006100009F060C022C0F801808189830E5F1F4FFE
:10062000420171E0A72EB12C16C062E0662E712C3B
:10063000600E711EF8018080918026FF03C06E2D30
:1006400070E002C06FEF7FEFC4012C870E9474043A
:100650005C0183012C852F7717C052E0652E712C29
:10066000600E711EF8018080918026FF03C06E2D00
:1006700070E002C06FEF7FEFC4012C870E94690415
:100680005C012C852068830123FD20C008C080E226
:1006900090E0B6012C870E947F04FA942C858F2D60
:1006A00090E0A816B90698F311C0F40127FD8591D2
:1006B00027FF81914F0190E0B6012C870E947F04B3
:1006C0002C85F110FA940894A108B108A114B10482
:1006D00061F7F1C0843611F0893649F527FF08C06B
:1006E000F80160817181828193810C5F1F4F09C085
:1006F000F80160817181882777FD8095982F0E5FC2
:100700001F4F4FE6B42EB22297FF09C090958095F7
:10071000709561957F4F8F4F9F4FF0E8BF2AA201E0
:100720002AE030E00E94AB04782E741845C085376B
:1007300031F43FEEB32EB2222AE030E025C099EF2B
:10074000B92EB2228F36C1F0803720F4883509F0F7
:10075000B5C00DC0803721F0883709F0AFC002C0A6
:1007600020E1B22AB4FE0BC084E0B82A08C0B4FE6F
:1007700009C0E6E0BE2A06C028E030E005C020E15E
:1007800030E002C020E132E0B7FE08C0F80160812D
:100790007181828193810C5F1F4F07C0F8016081D6
:1007A000718180E090E00E5F1F4FA2010E94AB04B8
:1007B000782E7418FFE7BF22B6FE0BC02EEFB222D0
:1007C0007E1438F4B4FE07C0B2FC05C08FEEB82228
:1007D00002C0A72C01C0AE2C8B2D90E0B4FE0DC042
:1007E000FE01E70DF11D2081203319F4E9EEBE2250
:1007F00009C0A394B2FE06C004C08678907000972A
:1008000009F0A3948B2C9924B3FC14C0B0FE0FC044
:10081000AF1428F4E72CEF0CEA18AF2C08C0E72C33
:1008200006C080E290E0B6010E947F04A394AF145A
:10083000C0F304C0AF1410F4FA1801C0FF2484FE02
:100840000FC080E390E0B6010E947F0482FE1FC0CB
:1008500081FE03C088E590E010C088E790E00DC0FD
:10086000C40186789070009791F081FC02C080E20C
:1008700001C08BE2B7FC8DE290E0B6010E947F04DC
:1008800006C080E390E0B6010E947F04EA947E14E3
:10089000C0F37A94F201E70DF11D808190E0B6017A
:1008A0000E947F047720A9F706C080E290E0B6019D
:1008B0000E947F04FA94FF20C1F737CEF60126810B
:1008C000378102C02FEF3FEFC9012C96E2E10C9473
:1008D0002505FC010590615070400110D8F7809506
:1008E00090958E0F9F1F0895FC01615070400190FC
:1008F0000110D8F7809590958E0F9F1F08950F9344
:100900001F93CF93DF938C01EB018B8181FF1BC081
:1009100082FF0DC02E813F818C819D812817390770
:1009200064F4E881F9810193F983E88306C0E885DE
:10093000F985802F0995009731F48E819F8101966A
:100940009F838E8302C00FEF1FEFC801DF91CF910D
:100950001F910F910895FA01AA27283051F12031F3
:1009600081F1E8946F936E7F6E5F7F4F8F4F9F4F43
:10097000AF4FB1E03ED0B4E03CD0670F781F891F85
:100980009A1FA11D680F791F8A1F911DA11D6A0F53
:10099000711D811D911DA11D20D009F468943F9106
:1009A0002AE0269F11243019305D3193DEF6CF0105
:1009B0000895462F4770405D4193B3E00FD0C9F7CB
:1009C000F6CF462F4F70405D4A3318F0495D31FD38
:1009D0004052419302D0A9F7EACFB4E0A69597958B
:1009E000879577956795BA95C9F700976105710561
:1009F00008959B01AC010A2E0694579547953795AB
:100A00002795BA95C9F7620F731F841F951FA01D04
:100A100008952F923F924F925F926F927F928F92A2
:100A20009F92AF92BF92CF92DF92EF92FF920F937D
:100A30001F93CF93DF93CDB7DEB7CA1BDB0B0FB687
:100A4000F894DEBF0FBECDBF09942A883988488844
:100A50005F846E847D848C849B84AA84B984C884DA
:100A6000DF80EE80FD800C811B81AA81B981CE0FD1
:100A7000D11D0FB6F894DEBF0FBECDBFED010895B6
:040A8000F894FFCF18
:100A840000000000000015001A1D04040405020003
:100A94000A040E100E011E000A040E1010110C00A0
:100AA400567A6469616C3A20257520636D20202094
:040AB400000D0A0027
:00000001FF
